:100000000C9461000C947E000C947E000C947E0095
:100010000C947E000C947E000C947E000C947E0068
:100020000C947E000C947E000C947E000C947E0058
:100030000C947E000C947E000C947E000C947E0048
:100040000C949D000C947E000C947E000C947E0019
:100050000C947E000C947E000C947E000C947E0028
:100060000C947E000C947E00000000002400270009
:100070002A0000000000250028002B0000000000DE
:1000800023002600290004040404040404040202DA
:100090000202020203030303030301020408102007
:1000A0004080010204081020010204081020000012
:1000B0000007000201000003040600000000000029
:1000C000000011241FBECFEFD8E0DEBFCDBF11E08E
:1000D000A0E0B1E0EAE3F4E002C005900D92A230A6
:1000E000B107D9F711E0A2E0B1E001C01D92AB3039
:1000F000B107E1F70E940C020C941B020C94000063
:100100008091000161E00E94B80168EE73E080E038
:1001100090E00E94E5008091000160E00E94B8013B
:1001200068EE73E080E090E00E94E5000895809121
:10013000000161E00E94790108951F920F920FB6AD
:100140000F9211242F933F938F939F93AF93BF935D
:100150008091060190910701A0910801B0910901D9
:1001600030910A010196A11DB11D232F2D5F2D375E
:1001700020F02D570196A11DB11D20930A018093F7
:10018000060190930701A0930801B09309018091A3
:10019000020190910301A0910401B0910501019623
:1001A000A11DB11D8093020190930301A09304014E
:1001B000B0930501BF91AF919F918F913F912F9186
:1001C0000F900FBE0F901F9018959B01AC017FB749
:1001D000F8948091020190910301A0910401B091E3
:1001E000050166B5A89B05C06F3F19F00196A11DDA
:1001F000B11D7FBFBA2FA92F982F8827860F911D79
:10020000A11DB11D62E0880F991FAA1FBB1F6A952F
:10021000D1F7BC012DC0FFB7F894809102019091F5
:100220000301A0910401B0910501E6B5A89B05C0AA
:10023000EF3F19F00196A11DB11DFFBFBA2FA92FE5
:10024000982F88278E0F911DA11DB11DE2E0880F08
:10025000991FAA1FBB1FEA95D1F7861B970B885ED3
:100260009340C8F2215030404040504068517C4F8C
:10027000211531054105510571F60895789484B52D
:10028000826084BD84B5816084BD85B5826085BD92
:1002900085B5816085BDEEE6F0E080818160808378
:1002A000E1E8F0E01082808182608083808181605B
:1002B0008083E0E8F0E0808181608083E1EBF0E022
:1002C000808184608083E0EBF0E0808181608083C6
:1002D000EAE7F0E0808184608083808182608083AF
:1002E0008081816080838081806880831092C100DA
:1002F0000895CF93DF93482F50E0CA0186569F4F51
:10030000FC0134914A575F4FFA018491882369F1C7
:1003100090E0880F991FFC01E859FF4FA591B49117
:10032000FC01EE58FF4FC591D491662351F42FB7CD
:10033000F8948C91932F909589238C9388818923AD
:100340000BC0623061F42FB7F8948C91932F909585
:1003500089238C938881832B88832FBF06C09FB706
:10036000F8948C91832B8C939FBFDF91CF9108954C
:10037000482F50E0CA0182559F4FFC012491CA01C9
:1003800086569F4FFC0194914A575F4FFA01349172
:10039000332309F440C0222351F1233071F024307B
:1003A00028F42130A1F0223011F514C02630B1F02C
:1003B0002730C1F02430D9F404C0809180008F77B9
:1003C00003C0809180008F7D8093800010C084B531
:1003D0008F7702C084B58F7D84BD09C08091B00045
:1003E0008F7703C08091B0008F7D8093B000E32FA2
:1003F000F0E0EE0FFF1FEE58FF4FA591B4912FB71D
:10040000F894662321F48C919095892302C08C91F5
:10041000892B8C932FBF0895CF93DF930E943E01C9
:100420000E949700C0E0D0E00E9480002097E1F396
:0A0430000E940000F9CFF894FFCFFE
:02043A000D00B3
:00000001FF
